:10100000F0BE03207D270000634800006348000015
:1010100063480000634800006348000000000000CF
:101020000000000000000000000000006348000015
:1010300063480000000000006348000063480000AF
:10104000252800003528000063480000592A0000C8
:1010500063480000634800006348000063480000E4
:10106000634800006348000063480000892A0000CC
:1010700063480000634800006348000063480000C4
:1010800063480000634800006348000063480000B4
:1010900063480000634800006348000063480000A4
:1010A0006348000063480000634800006348000094
:1010B00063480000634800000000000000000000DA
:1010C0006348000063480000634800006348000074
:1010D000634800006348000063480000652B00007F
:1010E00063480000634800006348000000000000FF
:1010F000000000006348000000000000634800009A
:10110000111900000400000004000000D7190000BD
:1011100013190000B1190000525B5D4D446657770A
:101120007E636A21313A3B6473622E347156424ABF
:101130005C3C7B2225292A4C494758362327375EB9
:101140004041515F6972793E7C28657D596F356EEB
:101150007024763F336C383D264E5A482B672F4516
:1011600030207561687432537A2C552D50784B5469
:101170004F4643606B6D39475C75783322576E5329
:10118000516C2C7348204F6A49313F723D2F2154D6
:1011900068715D246F746B7B5B2D3B25645E6163BE
:1011A0002A2339267D36504252585A692755655FA1
:1011B000402E4A663556416D293C767037774D385A
:1011C0004460624B434C3A287C32453E2B464E7A73
:1011D0003059347E677900004E4B62657E6A442246
:1011E000277D445F627D432651265F624326653733
:1011F00044266544434B58447A2B264F26285844AE
:101200005B3527496235446E277D7E6A4B275F2C0C
:1012100064657669636569643D00000070130000D1
:10122000000000007013000000000000000000003B
:101230002000000008000000020000000000000084
:101240000000000008000000030000000100000092
:101250002000000008000000020000000000000064
:101260000000000008000000030000002063686127
:101270006E6E656C3D205478506F7765723D2B38EB
:1012800064426D206170703D70757A7A6C652E686D
:1012900065780A006C120000090000007512000059
:1012A0001E000000636F7272656374696E636F7213
:1012B000726563747265636569766564202062791E
:1012C00074650000B412000009000000BD120000A7
:1012D00005000000734572724F6B20284352433D56
:1012E00028290000DA12000006000000E0120000C9
:1012F00001000000E11200000100000000000000F9
:1013000020000000000000000200000000000000BB
:1013100002000000000000000300000001000000C7
:10132000200000000C00000002000000000000008F
:101330000000000006000000030000002C204C51BB
:10134000493D00003C13000006000000290A6469C2
:10135000646E2774207265706C79202D2D2063686F
:10136000616E6E656C2077617320627573790A0017
:101370003030303130323033303430353036303751
:101380003038303931303131313231333134313537
:10139000313631373138313932303231323232331D
:1013A0003234323532363237323832393330333103
:1013B00033323333333433353336333733383339E9
:1013C00034303431343234333434343534363437E1
:1013D00034383439353035313532353335343535C7
:1013E00035363537353835393630363136323633AD
:1013F0003634363536363637363836393730373193
:101400003732373337343735373637373738373978
:101410003830383138323833383438353836383770
:101420003838383939303931393239333934393556
:10143000393639373938393930780B01003235329D
:10144000343233323232313230313931383137316E
:1014500036313531343133313231313236000000FA
:10146000F0B503AF2DE9E00F8B688A460969D0E932
:101470000069012B02D1012903D077E0012940F056
:10148000D480B9F1000F53D0DAF8141006EB090E2E
:10149000019300224B1C3146344602960D4615F945
:1014A000010BB0F1FF3FC6B229DC754505D0487885
:1014B0008D1C00F03F0C294602E04FF0000C7146F5
:1014C00006F01F0BDF2E07D9714508D011F8010B6C
:1014D00000F03F080D4605E04CEA8B160FE04FF098
:1014E0000008714648EA8C1CF02E06D371450FD0D7
:1014F00011F8010B00F03F060CE04CEA0B362946D0
:10150000013B17D0121B8E450A440C46C6D10BE096
:10151000002629464FF4E01000EA8B4040EA8C1088
:101520000644B6F5881FEBD14A46DDE901361AE0DC
:10153000002218E0019BB6F5881F02D14A46029EA0
:1015400011E0029E3AB14A4505D04A4505D2B0564F
:1015500010F1400F01DB304601E00020002200289E
:101560000CBF4A460646012B0CD19146B9F1000F3B
:101570000BD0A9F1010009F0030C032807D20020C9
:10158000324625E0DAE9060154E000203BE0ACEB0E
:1015900009030020B64632461478557804F0C0049A
:1015A0009678D178802C05F0C00408BF0130802CDB
:1015B00006F0C00408BF0130802C01F0C00108BF54
:1015C0000130802908BF013004320433E4D176466B
:1015D000BCF1000F17D0117801F0C001802908BFBD
:1015E0000130BCF1010F0ED0517801F0C00180290B
:1015F00008BF0130BCF1020F05D0917801F0C001A5
:10160000802908BF0130DAF80CE0A9EB0001714530
:101610000BD2B9F1000F15D0A9F1010109F0030CAB
:10162000032911D2002133462FE0DAF81C104A4674
:10163000DAF81800CB68314603B0BDE8000FBDE80A
:10164000F040184700213BE0ACEB09040021B04614
:1016500033461D785E789A7805F0C005D878802DDD
:1016600006F0C00508BF0131802D02F0C00208BF9E
:101670000131802A00F0C00008BF0131802808BF76
:10168000013104330434E4D14646BCF1000F17D0D5
:10169000187800F0C000802808BF0131BCF1010FAC
:1016A0000ED0587800F0C000802808BF0131BCF18E
:1016B000020F05D0987800F0C000802808BF0131E3
:1016C0009AF82000C21E18BF0246A1EB090000EBE9
:1016D0000E0100200C46DFE802F00802050200249B
:1016E000084602E0480801314C08451C013D08D07D
:1016F000DAE90602DAF80410126990470028F5D0FA
:1017000013E0DAE906014A46CB683146DAF804B05C
:10171000984750B9DAE906650134013C09D02A69D5
:101720003046594690470028F7D00120BDE80E0FFB
:10173000F0BD0020FAE7D4D4F0B503AF2DE9000FD7
:101740008DB0D1E9023BD1E900A6D1E9045C0321C7
:101750008DF830102021059100216B4A04910B92E5
:1017600003AA0A920891039006910293C3B1B3456C
:1017700088BFB346BBF1000F2DD0DAF80410026821
:101780005318802B00F2B280DAF80030A1B3024483
:1017900013F8014B01391471026801320260F5E758
:1017A000B44588BFB446BCF1000F14D0DAF8041079
:1017B00002685318802B00F29980DAF80030E34673
:1017C000002978D0024413F8014B013914710268E2
:1017D00001320260F4E74FF0000846450AD90AEBEF
:1017E000C8005AF838104268DDE90A03DB689847F8
:1017F00000287BD100207AE00298544601964FF0F1
:10180000010800F110094FF0000A6646029800EB4B
:101810008A0148680590087F8DF830008868049038
:10182000D1E9052062B1022A0CD0B04268D205EBA2
:10183000C002364B52689A4204D155F83000006815
:10184000012200E00022CDE90620C968D9F8000095
:1018500061B102290CD0B04252D205EBC0012B4A33
:101860004968914204D155F830000068012100E038
:101870000021CDE9081059F8100CB04240D255F8BB
:10188000301005EBC0004268084604A9904768BBC9
:10189000D84530D204EB0A00D0E90212DDE90A0390
:1018A000DB6898470AF1080A09F1200908F10108E4
:1018B0000028ABD01AE00DF110093446002605EBE4
:1018C000C60155F836004A684946904770B906F196
:1018D0000108D84512D20AEBC600D0E90212DDE9B0
:1018E0000A03DB68984700284646E8D001200DB07F
:1018F000BDE8000FF0BDA246019E6EE726466CE7EC
:10190000314600F0DAFCFEDE00110000AD220000DE
:101910007047E0B502AF0068802909D202687F2ACB
:1019200018D80244117101680131016000203DE0C6
:101930000022B1F5006F01924FF002020CD28B0928
:1019400062F39F118DF80510062161F35F138DF886
:10195000043028E0012029E00B46B1F5803F62F316
:101960009F130ED28DF806308B0962F39F13090B7B
:101970000E228DF8053062F31F118DF8041003223A
:1019800011E08DF80730F02343EA91438DF80430DD
:101990008B09090B62F39F1362F39F1104228DF8E8
:1019A00006308DF8051001A900F02AF802B080BDBC
:1019B000F0B503AF4DF8048D86B00068EC4691E8B1
:1019C00074416346614683E87441FFF7B5FE06B093
:1019D0005DF8048BF0BD006800F012B804C8C9B20D
:1019E00052003AB110F8023B023A8B42F9D1411E43
:1019F000023801E00020002100B9002108467047AC
:101A0000D0B502AF03689C18802C01D90120D0BD4D
:101A100042B1034411F8014B013A1C7103680133D0
:101A20000360F5E70020D0BD80B56F46017839B17D
:101A3000032902D14178012904D100F039FCFEDEEE
:101A400000214170064901220978C9B2002908BF66
:101A5000032202704270B1FA81F0400980BD00BFDC
:101A600094F1032080B56F46ADF50A7DD248402140
:101A7000DFF89CA701600AF105000121D0E84F2F93
:101A8000002A40F0A683C0E8421F002AF6D10AF1DE
:101A900004000121D0E84F2F002A40F0A783C0E8BE
:101AA000421F002AF6D1C5494B20DFF874C7DFF882
:101AB00074E7C1F8FC002AA901F10408002009908C
:101AC0002A905F2820D02A9D41461CF800401EF82D
:101AD000006001306A003AB111F8023B023AB342A9
:101AE000F9D14A1E023901E00021002209B1147027
:101AF000E7E77F2DE5D808EB450108F815604C7045
:101B00002A9901312A91DCE70DF12408DFF8181732
:101B100009224046FFF774FFA9487FAE0DF504790E
:101B2000022541687C9100687F90DFF80407DFF8A8
:101B3000FC168791CDE985167CA984916BA97095D7
:101B4000CDE96E59CDE96C50DFF8E8066B90404660
:101B5000FFF7F2FD994C4FF0010BDFF8DC16D4F8DB
:101B6000FC000024CDE96F9B6E9400F07F00CDE96E
:101B70006C546BADCDE98461DFF8C0166B912946DA
:101B80008DF8FC014046FFF7D7FD2AA88DF8C84123
:101B9000CDF8BC916E9005F12E00029005F12D005C
:101BA000019005F12800039005F13800059005F13A
:101BB0003000CDE96C89B0460026069005F114008E
:101BC000079005F12000CDF8AC9104909DF8C80174
:101BD000DFE810F00600D502D50222003B00090024
:101BE0008DF8CC611DE09DF8E001DFE810F0780190
:101BF000C902C8027E01070051004B009DF8E801B0
:101C0000810700F07B81032840F0BA829DF8E9014A
:101C1000012840F07581B3E29DF8CC01012800F065
:101C2000AF82DAF8100060B101685AE8042F8242EE
:101C300004D14AE80412002AF3D117E0BFF32F8F32
:101C4000EFE703208DF8CC0194E29DF8D801DFE89E
:101C500010F03900970296023D00060013009DF82F
:101C6000E40181071FD0032844D089E20221C1701A
:101C700070908DF8CCB11AE09DF8EC0180B103288A
:101C800073D07DE29DF8E401012840F0C68177E23F
:101C90009DF8EC0148B1032840F072827A9D43E13F
:101CA000DDE977015FE0779823E0799D3BE16C986F
:101CB00050F8041B02F004FD07988DF8D861749069
:101CC0006D987390ADF8DC61749875900698FFF785
:101CD000ABFE18B103208DF8D80193E04FF480706B
:101CE000ADF8D9010120000650D003988DF8E461C9
:101CF000779078909AF80600C0B218B1022800F0E8
:101D000079804FE202F070FC5FFA80F8B8F1000FC2
:101D100061D0B8F1010F6DD0B8F1020F40F03382FD
:101D200078982649006800680330C1F8F800254813
:101D30008AF807B0C0F800B002F00CFDCDE98401CC
:101D40004846022102F018F8DFF8F814484602F07D
:101D50002DF801990DF5FE7802988DF8E4B18DF813
:101D6000EC6178917790CDE979019AF8070000F05D
:101D70000300DFE810F0170204001400290005201A
:101D80008DF8D80103208DF8EC013BE00B48016889
:101D90008DF8D8B19DF8D90180F0010034E08AF8BF
:101DA0000760799806700748D0F8F8037A9900F030
:101DB000010008700AE000BF0C0500500C14004040
:101DC00060000010081000408AF807608DF8ECB140
:101DD0009DF8DA0187E702F001FC02F0BBFCCDE9D7
:101DE00084014846022101F0C7FFDFF85C14484631
:101DF00001F0DCFF04200DF5FE788DF8D8010320FA
:101E00008DF8E4010021022082B2022A01D10420CF
:101E1000B0E1ADF8C401ADF8C611709BDA78023AB2
:101E20008DF8CC21D2B2032A08D3DA78023A53FAD9
:101E300082F212798DF8CE21012200E00022000406
:101E40008DF8CD2101D00020FDE0D878032807D0FF
:101E5000DFF8FC13022813D13A203822D87034E07E
:101E600019796E988DF81012FFF7B8FD002808BF99
:101E70004846709903220078CA707099087128E06A
:101E800002381C1DC5B25DB126466E9816F8011BBE
:101E9000FFF7A4FD08B100782070013D3446F2E759
:101EA000709D0026E8783A2808D1DFF8A413281D91
:101EB000884206D0382202F044FD10B1E6490922DA
:101EC00001E00722E349901CE8707098043002F0AA
:101ED0006FFD07988DF8E06175906F987490DDE95B
:101EE00074017690ADF8E46177910598FFF79CFD59
:101EF00008B103203BE17A96769879908DF8E961F4
:101F00009AF808000121C0B2022808BF0321022864
:101F10008DF8E8118DF8E91101D1042027E1069D23
:101F20008DF8EC6179957A95002100208DF810B23A
:101F3000012906D019F8012001310BFA02F21043F1
:101F4000F6E708B1C54908609AF8060000F00300FA
:101F5000012800F00381B0BB02208AF8060002F0DD
:101F6000F9FBCDE984014846022101F005FFBC4997
:101F7000484601F01BFF2868A84900680330C1F8F3
:101F8000F800AF4801464FF48040C1F80003D1F893
:101F9000F80140F48010C1F8F8019AF80700C0B2C7
:101FA000012810D103208AF80700A548C0F804B022
:101FB00002F0D0FBCDE984014846022101F0DCFEAD
:101FC0004846A849C8E002F00FFBC5B2002D00F05A
:101FD000B780012D00F0C280022D40F0E6809848C5
:101FE0004FF000618AF808B0C0F8FC12C0F824B0C5
:101FF00002F0B0FBCDE984014846022101F0BCFEAD
:102000009949484601F0D2FE48468DF810B202F0D8
:10201000CDF98DF8ECB18DF8E4619AF80800012251
:10202000C1B2012908BF032201298DF8E42101D1A1
:1020300006209CE06FF0030151FA80F0B0FA80F0C6
:102040008DF8E0B1400908906C98016801394A1C8C
:1020500001D00160FAE70224002189944546CDE9C8
:1020600087187CAECDE9854180498491DFF80082F4
:102070008049CDF808828196809104997F919DF8DE
:10208000CC116C984A1E18BF012201297B497D9210
:10209000794A08BF11467C914946FFF74DFBBDF8D0
:1020A000C401774A01284FF0020008BF03207D9049
:1020B000BDF8C611734808BF104627F82E1C724998
:1020C0008994CDE987458691032185916F49849153
:1020D0006F497C908291A7F12E016C98CDE98081A7
:1020E00049467F96A846634C0026FFF725FB9DF8DE
:1020F000CD0190B19DF8CE0187A981E8400907F88C
:10210000190C6C986349CDE985B68491A7F1190142
:1021100080947F914946FFF70FFB6C9802225E493D
:10212000FFF76EFC089800283FF4C1AD6C9821229F
:102130005A49FFF765FC6C9802C802F0C1FAB6E58F
:1021400002F04CFA02F006FBCDE984014846022178
:1021500001F012FE5249484601F028FE48468DF82B
:1021600010B202F023F903208DF8EC0105208DF860
:10217000E00105208DF8C80102F07BFB26E5FEDEBC
:1021800000F096F8FEDE02F0E5FA84ACCDE98401B9
:102190000021204601F0F0FD2C49204601F006FE0A
:1021A000404610E001F0CEFFFEDE02F0D3FA84AC30
:1021B000CDE984010021204601F0DEFD39492046A9
:1021C00001F0F4FD2846214602F02AFA02F064FAF2
:1021D000FEDEBFF32F8F02F0BDFA2AACCDE92A0153
:1021E0000021204601F0C8FD0A490BE0BFF32F8F04
:1021F00002F0B0FA2AACCDE92A010021204601F014
:10220000BBFD0549204601F0D1FD02F02BFBFEDEAF
:1022100098F1032061000000560000000C140040FB
:10222000771100001811000010120000AB2600000A
:102230002C1200001C120000114500009412000036
:10224000081000405800000057000000590000002E
:10225000D8110000A4120000AB12000080E100E0E1
:102260005A0000005B0000005D000000C412000086
:10227000611400002F26000070130000D41200002B
:10228000D5120000D8120000FC120000E412000079
:1022900081250000441300004C1300004E13000081
:1022A0005C0000005E00000002F0DDBA0068FEE79E
:1022B00080B56F4600F006F8FEDE80B56F4600F090
:1022C00001F8FEDE80B56F4602F03EFAFEDED4D4A1
:1022D000F0B503AF2DE9000F83B0D0F800E09246CF
:1022E000BD680A461EF001014FF02B0B01EB0506FD
:1022F00008BF4FF4881B1C4680465FEA4E7103D42A
:102300004FF0000A002254E0BAF1000F0BD0AAF1FE
:1023100001010AF0030C032907D200211346BCF186
:10232000000F2BD142E0002140E08DE87000ACEBC3
:102330000A060021914613461A785D78987802F0D3
:10234000C002DC78802A05F0C00208BF0131802A73
:1023500000F0C00008BF0131802804F0C00008BFB1
:102360000131802808BF013104330436E4D1DDE9AE
:1023700000454A46029EBCF1000F17D0187800F0C5
:10238000C000802808BF0131BCF1010F0ED0587881
:1023900000F0C000802808BF0131BCF1020F05D059
:1023A000987800F0C000802808BF013106EB0A00D1
:1023B000461AD8F80800012818D1D8F80C90B14571
:1023C00014D95FEA0E702AD40292A9EB060198F89C
:1023D000202000208946032A08BF0122DFE802F0FE
:1023E000490245024FF00009084642E0404659467E
:1023F000534600F09EF828B10126304603B0BDE8F0
:10240000000FF0BDD8F81C102A46D8F81800CB6889
:10241000214603B0BDE8000FBDE8F0401847D8F8EA
:10242000040059460296012601903020C8F80400A5
:10243000534698F820000090404688F8206000F04D
:1024400078F80028D9D198F82020AA460298032AC3
:1024500008BF0122A9EB000100200D46DFE802F0D1
:102460003A0237020025084634E0480801314FEAB5
:102470005109461C013E08D0D8E90602D8F80410DC
:10248000126990470028F5D0B6E7029A40465946AF
:102490005346D8F8046000F04CF80028ACD1D8E9D5
:1024A00006012A46CB68214698470028A4D109F1A5
:1024B0000105D8E9069834460126013D2FD0D8F809
:1024C00010204846214690470028F6D095E7480856
:1024D00001314D08461C013E08D0D8E90602D8F863
:1024E0000410126990470028F5D085E7D8E9060264
:1024F0002146D3685246D8F80440984700287FF414
:102500007BAFD8E9069A01350126013D09D0DAF8FA
:1025100010204846214690470028F6D06DE7002657
:102520006BE70098002688F820000198C8F804009E
:1025300063E7F0B503AF4DF804BD1C4615460646EB
:10254000B1F5881F08D0D6E906021269904718B184
:1025500001205DF804BBF0BD4DB1D6E9060122466D
:10256000CB6829465DF804BBBDE8F0401847002061
:102570005DF804BBF0BD80B56F46FFF7A3FEFEDE3D
:10258000F0B503AF4DF804BDA2B0068802AD0C460D
:10259000802106F00F0000F157020A2838BF00F131
:1025A0003002284602F057FA0020B0EB161F28D060
:1025B000310901F00F0101F157020A2938BF01F179
:1025C0003002B0EB162F8DF886201DD0300A00F0B7
:1025D0000F0000F157010A2838BF00F13001002038
:1025E000B0EB163F8DF8851011D0300B00F157017C
:1025F0000A2838BF00F130018DF884107C200421B6
:1026000007E07F20012104E07E20022101E07D20FF
:102610000321009141F238412B18C0F200012046FD
:102620000222FFF755FE22B05DF804BBF0BD80B575
:102630006F468CB00A460178642915D348F21F50C2
:10264000C5F2EB10A1FB00036FF063005B0903FB15
:10265000001041F27031C0F20001C0B231F8100038
:10266000ADF82D00242003E00A2906D226200B46CF
:1026700003F1300102AB195408E041F27030C0F2AE
:10268000000030F81100ADF82D002520C0F1270121
:10269000009102A90B1841F270311046C0F20001FE
:1026A0000022FFF715FE0CB080BDB0B502AFA2B09E
:1026B00000680DF1080E8C468123002200F00F0106
:1026C00001F157040A2938BF01F130040EEB030170
:1026D000B2EB101F01F8024C30D0040904F00F04D3
:1026E00004F157050A2C38BF04F13005B2EB102F66
:1026F00001F8035C27D0040A04F00F0404F1570525
:102700000A2C38BF04F13005B2EB103F01F8045C2D
:102710001ED0040B043B04F00F0404F157050A2CEF
:1027200038BF04F1300501F8055C010CB2EB104F25
:102730000846C3D1581E81280ED31CE0981E013BC9
:10274000812809D317E0D81E023B812804D312E068
:10275000181F033B81280ED2C3F18101009141F281
:1027600038410EEB0003C0F2000160460222FFF781
:10277000AFFD22B0B0BDFFF7FEFEFEDE80B56F46B6
:102780001B481D4A016841F0807101601948002111
:102790004160016811400131016018480121C0F811
:1027A0001015016016488160016016481649091A23
:1027B00021F0030102F09EF914481549091A21F08D
:1027C0000302144902F0F6F802F04FF812484FF4F1
:1027D0008A51124C124D01600161AC4202D201CC0F
:1027E0008047FAE7FFF760FDFFF73CF9FEDE00BF28
:1027F000FCED00E0001000E0FEFFFF0008000040DC
:1028000000B0004000F00320ACF10320ACF1032045
:102810002CF203200C4B000008050050FC4A00007D
:102820000C4B000080B56F4601F0A0FCBDE8804075
:1028300001F0CABCF0B503AF2DE9C00B01F08AFF6F
:102840006C46CDE900012046042101F095FA794952
:10285000204601F0ABFA784A906B000605D00020C4
:102860009063D2F80402400406D41068000607D032
:102870004FF0040810461BE091464FF002081AE0A2
:10288000104650F8481F090602D04FF000080FE02C
:10289000104650F80C1F090602D04FF0010807E05F
:1028A000104650F86C1F090600F0C0804FF0030876
:1028B00091460021016001F04DFF6E460446CDE9CE
:1028C00000010D463046032101F056FA5B493046BF
:1028D00001F06CFA28880C22411C6FF31F3022543F
:1028E00030462980564901F061FADFE808F00372AA
:1028F0002B482100DDE9000100250A88531C6FF3F5
:102900001F3285540B8001F025FF6C46CDE9000194
:102910002046022101F030FA4E49204601F046FAE5
:102920004FF000600421C9F808024648857161E053
:10293000DDE9000104240A88531C6FF31F3284541C
:102940000B8070E0DDE9000102240A883D4D531C34
:102950006FF31F3284540B80A879000666D101F012
:10296000F9FE6C46CDE900012046022101F004FA8F
:102970003649204601F01AFA0120A87153E0DDE93A
:102980000012032013885C1C6FF31F33C8542D49B9
:1029900014808A79D2B2022A48D14FF48042C9F811
:1029A0000422D9F8002122F48012C9F800214FF046
:1029B0000062C9F8082200228A71087201F0CAFE7A
:1029C0006C46CDE900012046022101F0D5F91E49EF
:1029D00026E0DDE9000101240A88531C6FF31F3251
:1029E000845418480B808179C9B2012904D0022986
:1029F0001CD10221017216E0C179C9B2012915D199
:102A00000021C9F86C1081710221C17101F0A2FE90
:102A10006C46CDE900012046022101F0ADF90C49D8
:102A2000204601F0C3F9BDE80C0BF0BD01F08AFBB4
:102A3000FEDE00BF48000000001100404900000019
:102A40004E00000098F103204D0000004B000000F4
:102A50004C0000004A000000DCB504AF01F07AFE33
:102A60006C46CDE900012046042101F085F90449B6
:102A7000204601F09BF9034800210160DCBD00BF46
:102A80004700000018310040DCB504AF2F48016852
:102A9000C90741D1C16BC90722D000212F4CC163A6
:102AA0002D490A88931C013204EA03332C4C23601D
:102AB0000A8091B20C22B1FBF2F202EB4202A1EBCE
:102AC000820103290CD8DFE801F00207020721493F
:102AD0004FF480724A6003E01E494FF480720A602E
:102AE000016CC9071FBF002101644FF40031C0F819
:102AF0000412416CC9071FBF002141644FF48021BB
:102B0000C0F80412816CC9071FBF002181644FF413
:102B10000021C0F80412DCBD01F01CFE6C46CDE9BA
:102B200000012046002101F027F90949204601F063
:102B30003DF908484FF480510160402101604FF495
:102B40008071416001F08EFEFEDE00BF04B10040E6
:102B5000460000000805005000F0032000F0FF00D0
:102B600040B50040F0B503AF2DE9000F93B001F080
:102B7000F1FD0AACCDE90A010421204601F0FCF880
:102B8000DFF82C1E204601F011F9D84AD2F8540182
:102B9000000604D002F5AA704FF007093DE0104688
:102BA00050F8FC1F090602D04FF0080935E0D2F8B2
:102BB0002401000604D002F592704FF003092CE0C6
:102BC000D2F85801000604D002F5AC704FF00409A9
:102BD00023E0D2F85C01000604D002F5AE704FF09D
:102BE00005091AE0D2F82C01000604D002F596700F
:102BF0004FF0000911E0D2F83801000604D002F5C8
:102C00009C704FF0010908E0D2F81001000600F0B6
:102C10006B8402F588704FF0020900219246016032
:102C200001F098FD0AAE0446CDE90A010D46304692
:102C3000032101F0A1F8DFF87C1D304601F0B6F861
:102C400028880C22411C6FF31F3022543046298003
:102C5000DFF8641D01F0AAF80820DFE809F0050993
:102C60000B070F110D13140000200CE003200AE0E5
:102C7000012008E0022006E0062004E0042002E033
:102C8000052000E00720DDE90A121388DFF82C8D0B
:102C90005C1C6FF31F33C854148098F80200811E27
:102CA000CAB2032A28BF0121C9B2012911D00229C1
:102CB00014D1DFE819F009000E01AE00BA00470098
:102CC0001F01A401F500AB01DFF8F40C00214181E4
:102CD000E0E1B9F1070F08BF002802D001F084F845
:102CE000FEDE01F097F80005F8D5012088F8020013
:102CF00001F030FD0AACCDE90A010221204601F0C5
:102D00003BF8DFF8C01C204601F050F898F80000AE
:102D1000002800F0BF8198F80100002800F0BA8177
:102D200098F80200002800F0B581042088F802001D
:102D30000020A8F8000013B0BDE8000FBDE8F04087
:102D400001F0B8B8DFF8780C40890028C6D1684E89
:102D500001220025D6F800905FFA89F0C109B2EB94
:102D6000D01F0C4618BF0224B5EBD01F08BF0C467D
:102D7000D6F804A0B368022CF068D9B241EA002169
:102D80000991D6F810E07169B269F6695FFA8EFCB4
:102D90004CEA012BD2B242EA06220892CDF81C90EE
:102DA00040F04B818DF83050CDE90A555546DDE9AC
:102DB000089601F0CFFC0DACCDE90D0100212046B5
:102DC00000F0DAFFDFF8001C204600F0EFFF079864
:102DD000214601F001F92846214601F0FDF8DFF80F
:102DE000EC5B30462146A84758462146A84748464E
:102DF0002146A8473D490120086501F0ABFC0AAC1B
:102E0000CDE90A010221204600F0B6FFDFF8701E6E
:102E10003DE101F09FFC0AACCDE90A010221204608
:102E200000F0AAFFDFF85C1E31E1DFF86C6E7089FC
:102E3000012800F0218102287FF450AFD14601F033
:102E400089FC0AACCDE90A010221204600F094FF7A
:102E5000DFF8341E204600F0A9FFB089002800F0FA
:102E60001D81234DD5F880014030C5F88001B4891B
:102E7000412CC0F0168101F06DFC0AACCDE90A01CD
:102E80000221204600F078FFDFF8001E204600F007
:102E90008DFF4020214601F09FF8B08940381AE1AB
:102EA00000F0B8FFC10500F1D480800540F1E5864F
:102EB00001F050FC0AACCDE90A010221204600F0E5
:102EC0005BFFDFF8E81D204600F070FF0848002196
:102ED000CFE001F03FFC0AACCDE90A010221204617
:102EE00000F04AFFDFF8A81DD1E000BF04700240E7
:102EF00080740240DAF86854CAF8685415F0040681
:102F000008D0DFF8940D0078C0B202287FF4E6AE56
:102F100000F0E8FFA8072AD501F01CFC0AACCDE9B7
:102F20000A010221204600F027FFDFF8841D204619
:102F300000F03CFF01F00EFC0AACCDE90A010221D1
:102F4000204600F019FFDFF86C1D204600F02EFF30
:102F5000DFF8440D01210170DFF8400D8188C08841
:102F600089B280B288421EBFD348802101606EB111
:102F700001F0F0FB0AACCDE90A010221204600F085
:102F8000FBFEDFF8341D204600F010FF680318D563
:102F9000CA48866A804601F0DDFB0AACCDE90A0129
:102FA0000221204600F0E8FEDFF8101D204600F068
:102FB000FDFE06F07F00214601F00EF80020C8F863
:102FC000280028030DD501F0C5FB0AACCDE90A01A4
:102FD0000221204600F0D0FEDFF8E41C204600F07D
:102FE000E5FE280756D501F0B5FB0AACCDE90A018C
:102FF0000221204600F0C0FEDFF8C81C47E013B0F5
:10300000BDE8000FBDE8F04000F06CBF01F0A2FB8E
:103010000AACCDE90A010221204600F0ADFEDFF83E
:10302000801C204600F0C2FEDFF86C0C41780229BB
:1030300080F02386002141702CE0C9F34112002A60
:1030400051D0022A4CD0012A7FF4ACAE4FF48072EA
:103050004AE001F07FFB0AACCDE90A0102212046DB
:1030600000F08AFEDFF83C1C204600F09FFE9348EB
:103070000121C0F8AC100DE001F06CFB0AACCDE909
:103080000A010221204600F077FEDFF8E81C204606
:1030900000F08CFE13B0BDE8000FF0BD0020708181
:1030A000F8E701F057FB0DF12808CDE90A010221EC
:1030B000404600F061FEDFF8B81C404600F076FEA6
:1030C0002046414600F088FF00F0EAFF04F07F0050
:1030D000C5F884010020B0810120C9F80000D9E7BB
:1030E0004FF4007200E0002209F00F06032E3FF6B5
:1030F00059AE04F00104049306940023DFE806F0BF
:103100000A0205084FF4803304E04FF4003301E075
:103110004FF4403342EA0304C4F30122260A1C0C94
:10312000012A059337D00396002A069E7FF43AAE13
:103130005FFA8AF255460C2ACDF808B000F25382A5
:10314000DFE812F00D0035015102190151020601AC
:10315000BE00E70052016401AB019801A100002EFE
:1031600000F041820998000402BF089880B202284A
:1031700040F03982022C00F01182012C00F01B82F9
:10318000002C40F030820298000440F02C824FF076
:10319000000E04204EE106995FFA8AF0049A554623
:1031A00022283AD0DDF82090212821D0202808BFFD
:1031B000002948D0059A002406F00300ADF84040ED
:1031C0000F94CDE900B940EA1220099E2A4641EA4F
:1031D000002111A8334601F0D7FA9DF844000228D7
:1031E00040F022828DF830400320CDE90A4429E2E4
:1031F0000029DFD0012CDDD10998000404BF1FFA9B
:1032000089F00728D6D11FFA8BF0B0F5807F28BF50
:103210004FF0000CCED2022027E0DDF820900029EC
:10322000C8D1012C08BF5FEA0940C3D1099880B218
:1032300003289CBF1FFA8BF0FF28BBD862F3082C31
:10324000C2F3400011E0012CB4D10998000404BF7E
:103250001FFA89F00728ADD11FFA8BF0B0F5807FF7
:1032600028BF4FF0000CA5D203208DF82A000F983C
:10327000ADF828C0CDF82B00BDF84000ADF82F0008
:103280000120099EDEE1002E00F0AD81022C40F00D
:10329000AA810998000402BF089880B2022840F071
:1032A000A281029801F0A7FAC2B2022A00F09B8123
:1032B00000F0010E0A20BDE004E200E0807402404C
:1032C000002E00F09081002C40F08D8101F0A8FAD2
:1032D000C1B20C2900F087814FF0FF3151FA80F222
:1032E000062A00F2808104210220DFE812F00700A4
:1032F0005201A3007C017C016E0178010498000654
:1033000004BF02985FEA004040F06D81012100F0A7
:10331000A4BC56EA040140F0668101F081FAC0B213
:103320000C2800F06081032800F02981022800F0B9
:103330002881069E0128554640F0558104980006D4
:1033400004BF02985FEA004040F04D8101211EE178
:10335000002E40F04881099880B27F2800F2438116
:10336000002C40F04081089802990843000440F086
:103370003A8105205CE0002E40F035810898000479
:1033800040F03181099880B2002800F0DD800228E9
:1033900000F0BF80012808BF002C40F02481029873
:1033A000000440F020814FF0000E082042E0002E83
:1033B00040F01981032C00F016810898000440F0B9
:1033C0001281099880B2002800F0CD80012808BF42
:1033D000002C40F008810298000440F004814FF076
:1033E000020E0020002125E0002E00F0FC8008984D
:1033F00080B2012808BF002C40F0F580099802999E
:103400000843000440F0EF80012013E0002E40F05C
:10341000EA80099880B2FF2800F2E580002C40F095
:10342000E280089802990843000440F0DC800620FE
:10343000DDF810E0049AC9B2120642EA01415FFACF
:103440008EF241EA02210844CDF8290000200299B9
:103450008DF828000898C1EA0040CDF82D009DF8AD
:103460002A00BDF82810BDF82F80DDF82B4041EA76
:10347000004632E1002E40F0B680012C40F0B380CF
:10348000089A120401BF0002090208435FEA0040E3
:1034900040F0A98009200499CCE7002E00F0A38019
:1034A000029884F00103002180B2B0F5807F4FF0D4
:1034B000000038BF0120099A92B21A43089B9BB2C0
:1034C00083F001031A43B2FA82F25209104008BF96
:1034D0008646002800F08780002203200492002204
:1034E000029200220892A5E7DFF8AC070078C0B28C
:1034F00001287FF4CFADDFF8A4078188C08889B2A6
:1035000080B288423FF4C6AD92464FF00609FFF7FD
:1035100087BB44EA0E00000665D16FF0020050FA46
:1035200081F24FF0020E0820032AFFF483AF069EBB
:10353000CAB2012A3FF47EAF5546022A53D14FF05A
:10354000020E0820022175E7022C4CD1029801F0EE
:1035500052F90491C1B2022945D000F001014FF0A7
:10356000010E082066E7022C3DD1029801F043F9D4
:10357000C2B2022A37D000F0010E00205AE7022121
:1035800005E0069E5FEA0B4055462CD1002107203E
:1035900064E30298000426D100215EE3029801F062
:1035A0002AF90491C1B202291DD000F001014FF0A7
:1035B000010E04203EE7029880B2B0F5807F12D25F
:1035C000714604204FF0020E34E70498000604BF51
:1035D00002985FEA004006D1022002212AE7029801
:1035E000000400F0398303982A460599DDF808B0F5
:1035F00000F00300CDF800B040EA1120DDF8209083
:10360000CDF8049046EA0021099E11A8334601F046
:10361000BBF89DF84400022806D100208DF8300048
:10362000CDE90A0003200DE01198CDF83500BDF872
:103630004800ADF839000D980A90DDF83700CDF854
:103640002B00022003283FF4B4AB9DF82A10BDF8EC
:103650002820DDF82B4042EA0146E0B3DFF8385677
:10366000012827D06878022858D104F47F00C6F3D7
:103670000745B0F5003F69D106F47F40B0F5807F83
:1036800040F0A68101F066F80AAECDE90A010221F8
:10369000304600F071FBDFF83C16304600F086FB48
:1036A0002846314600F098FC2046314600F097FC51
:1036B000FFF7A0BB687802283CD1300652D001F059
:1036C00049F80AACCDE90A010021204600F054FB7C
:1036D000DFF80816ADE2BDF82F8026F07F404FEAF4
:1036E000142A4FEA1049C0F30720DFE810F00B005E
:1036F000E2008B00CA007300F8001E01D6004B01E7
:103700007F00560101F026F80AACCDE90A0100213C
:10371000204600F031FBDFF854168AE201F01AF877
:103720000AACCDE90A010021204600F025FBDFF8B4
:1037300098157EE201F00EF80AACCDE90A010021ED
:10374000204600F019FBDFF8901572E201F002F854
:103750000AACCDE90A010021204600F00DFBDFF89C
:103760006C1566E26FF0010050FAA6F0C1B20229B2
:1037700028BF0220C6F30744C0B2002800F07781BA
:10378000012800F0418100F0E5FF0AADCDE90A0112
:103790000221284600F0F0FADFF84415284600F030
:1037A00005FB04F00100294600F016FCC6F30020DA
:1037B000294600F011FC00F0CDFF0AACCDE90A016A
:1037C0000221204600F0D8FADFF81815204600F054
:1037D000EDFA12E100F0BEFF0AACCDE90A010021CA
:1037E000204600F0C9FADFF8501522E200F0B2FFDF
:1037F0000AACCDE90A010021204600F0BDFADFF84D
:10380000F81416E200F0A6FF0AADCDE90A01022184
:10381000284600F0B1FADFF82815284600F0C6FA6D
:103820004046294600F0D8FBE0B2042800F2188296
:10383000DFE810F00500B501C9011602AA0100F089
:1038400089FF0AACCDE90A010221204600F094FA72
:10385000DFF80015204600F0A9FA5046214600F096
:10386000BBFB5FEA0A6000F0E98100F073FF0AAC7D
:10387000CDE90A010021204600F07EFADFF8D814D5
:10388000D7E100F067FF0AACCDE90A01002120462C
:1038900000F072FADFF8A414CBE100F05BFF0AAC91
:1038A000CDE90A010021204600F066FADFF8501445
:1038B000BFE100F04FFF0AACCDE90A01022120462A
:1038C00000F05AFADFF89C14204600F06FFA01204D
:1038D000214600F081FBDFF890040121B5E100F002
:1038E00039FF0AACCDE90A010221204600F044FA72
:1038F000DFF83014204600F059FA4846214600F01F
:103900006BFBE5494878002800F01F81012800F092
:10391000BF8000F01FFF0AACCDE90A01002120465C
:1039200000F02AFADFF8001483E100F013FF0AAC7C
:10393000CDE90A010221204600F01EFADFF8C41387
:10394000204600F033FA4846214600F045FBD248B5
:103950004078002800F00D81012800F0B180CE48A9
:10396000B9F1000F00F03A81C078484545D000F029
:10397000F1FE0AACCDE90A010021204600F0FCF975
:10398000E14956E100F0E6FE0AACCDE90A0100216A
:10399000204600F0F1F9D9494BE100F0DBFE0AAC1A
:1039A000CDE90A010021204600F0E6F9D14940E1C5
:1039B00000000000010000004500000022F203208A
:1039C00098F103200300000007000000DF3F000023
:1039D00000F0C0FE0AAECDE90A010221304600F037
:1039E000CBF9BB49304600F0E1F92846314600F0FA
:1039F000F3FA2046314600F0EFFA13B0BDE8000FAD
:103A0000BDE8F04000F046BB00F0A4FE0AACCDE9F2
:103A10000A010221204600F0AFF9B349204600F028
:103A2000C5F9688900287FF459A901266E8100F044
:103A300091FE0AACCDE90A010221204600F09CF972
:103A4000AA49204600F0B2F9974908F10300C1F8ED
:103A500080020720C1F884028E480146D0F8FC019C
:103A600040F00200C1F8FC018E64FFF713BB00F0C8
:103A700071FE0AACCDE90A010221204600F07CF972
:103A80009B49204600F092F908F103000721DCE091
:103A9000B9F1000F00F0B580887848453FF4FAAAE4
:103AA000012081F80290487000F054FE0AACCDE984
:103AB0000A010221204600F05FF99C49FFF7E7BAAE
:103AC000B9F1000F99D0B9F1010F40F0A880724808
:103AD0000546867800F03EFE0AACCDE90A010221D7
:103AE0004FF00209204600F047F98949204600F0CE
:103AF0005DF96D494FF001080F2085F80380AE7025
:103B000085F801900E46C1F890000920C1F8940094
:103B10000020C86200F01EFE0AACCDE90A010221B5
:103B2000204600F029F97B49204600F03FF90A20A1
:103B300021460A2500F050FA7748C6F89401554806
:103B4000C6F89851C0F8048057E7B9F1000F3FF468
:103B5000A1AA012081F80290487000F0FBFD0AAC98
:103B6000CDE90A010221204600F006F97149FFF76C
:103B70008EBA00F0EFFD0AACCDE90A010021204623
:103B800000F0FAF8664954E000F0E4FD0AACCDE933
:103B90000A010021204600F0EFF86A4949E000F0F0
:103BA000D9FD0AACCDE90A010221204600F0E4F873
:103BB0006649204600F0FAF8B8F1120F28BF4FF01E
:103BC0001208634840E000F0C5FD0AACCDE90A01E7
:103BD0000121204600F0D0F85B492AE006468578AE
:103BE00000F0B8FD0AACCDE90A010221204600F040
:103BF000C3F84649204600F0D9F80120B57070702E
:103C0000FBE60020487000F0A5FD0AACCDE90A01F2
:103C10000221204600F0B0F84549FFF738BA00F01D
:103C200099FD0AACCDE90A010021204600F0A4F874
:103C30003A49204600F0BAF8FFF7DCB84748B8F137
:103C40004B0F28BF4FF04B08414613B0BDE8000FA3
:103C5000BDE8F04000F0C6B903210220FFF7EABB3F
:103C600000F078FD0AACCDE90A010021204600F001
:103C700083F83B49204600F099F800F097F9FEDE02
:103C80002E000000390000002F000000300000006E
:103C90003A0000000470024098F10320ACF10320C8
:103CA00006000000040000008074024005000000CF
:103CB0003300000034000000350000003600000032
:103CC00037000000380000002A0000002B00000030
:103CD0002D0000002C00000023000000290000003F
:103CE000240000002500000027000000280000003C
:103CF0002600000008000000220000002100000053
:103D00002000000015000000180000001B0000004B
:103D1000190000001A00000014F203201700000030
:103D20001600000010000000110000001400000048
:103D300013000000120000001F0000001E00000021
:103D4000090000000F0000000C0000000B00000044
:103D5000B4F103200D0000000E000000C6F10320A6
:103D60000A0000001D00000020F203201C000000DB
:103D70003100000032000000F0B503AF4DF804BD83
:103D8000094A1268D0E90034258892096E1C6FF345
:103D90001F3559552680D0E9003118465DF804BB1F
:103DA000BDE8F04000F09AB9041000E0F0B503AFB0
:103DB0004DF804BD8AB27F2A0AD3D0E9003441F01D
:103DC000800125886E1C6FF31F355955D109268057
:103DD000D0E9002003885C1C6FF31F33D1540480AA
:103DE0005DF804BBF0BDD4D4E0B502AF00F092F9A9
:103DF00000F0B0FC6C46CDE9000120460021FFF741
:103E0000BBFF03492046FFF7D1FF00F02BFDFEDE8C
:103E100043000000F0B503AF2DE9F00B2248D0F8C5
:103E20000080C0F8008000F095FC01AC0546CDE9AB
:103E300001010E4620460321FFF79EFF1B49204645
:103E4000FFF7B4FF30880A22411C6FF31F302A5459
:103E5000204631801649FFF7A9FF029E40F6FF7108
:103E600027F81A8C358828466FF31F3088420DD109
:103E7000019CA7F11A09012204F6FF71484600F0DF
:103E80007BFC09F101002146012204E00199022294
:103E90000144A7F11A0000F06FFCA81C30804046D6
:103EA00004B0BDE8000BF0BD007402404200000009
:103EB00062000000DCB504AF08480121016000F099
:103EC00049FC6C46CDE9000120460221FFF754FF72
:103ED00003492046FFF76AFFDCBD00BF04750240BE
:103EE00041000000F0B503AF2DE9C007DFF8A4A042
:103EF000BAF80450BAF80600401B01041CD084B282
:103F00003F2C28BF3F2454FA85F081B2E8B2B1F5C6
:103F1000807F13D9DAF80090C0F58076DFF87880DA
:103F200009EB00013246404600F042FDA11B08EBC0
:103F300006008AB2494606E0012625E0DAF80010BC
:103F400022460144144800F033FD2819AAF8040061
:103F500020064FF0010617D000F0FCFB6D46CDE9BE
:103F6000000128460221FFF707FF0C492846FFF70A
:103F70001DFF2046294600F02FF809480649016038
:103F8000446008480660022607480670BDE80C0732
:103F9000F0BD00BFACF1032000C0032040000000D2
:103FA000287602400C70024098F10320E0B502AF81
:103FB00000F0B0F800F0CEFB6C46CDE900012046E1
:103FC0000021FFF7D9FE03492046FFF7EFFE00F07E
:103FD00049FCFEDE3D000000C0B200F069B880B2CE
:103FE00000F066B8F0B503AF4DF8048D82B0234EF3
:103FF0008046708990BB234C88B20D4640280AD970
:10400000206820F004002060A5F14000B08102206B
:104010004025708104E000F043F80220C6F80A0051
:1040200000F098FB6E46CDE9000130460221FFF713
:10403000A3FE15493046FFF7B9FE28463146FFF783
:10404000CBFF124905F07F0048601148C1F800809D
:104050000121215002B05DF8048BF0BD00F07AFB25
:104060006C46CDE9000120460021FFF785FE04499A
:104070002046FFF79BFE00F0F5FBFEDE98F10320E3
:104080003B000000007202403C000000007602404D
:1040900004FEFFFF0148012101607047507002409B
:1040A0000248016841F0040101607047007202405B
:1040B000F0B503AF4DF804BD0246D1E900031C88FA
:1040C0000626651C6FF31F3406551D80D1E90001DB
:1040D0005DF804BBBDE8F04000F000B8F0B503AFF8
:1040E0004DF804BD0C880023661C42F080056FF378
:1040F0001F34B3EBD21F08BF02F07F05B3EBD21F12
:1041000005554FEAD21534462A460E80ECD15DF8AB
:1041100004BBF0BDDCB504AF08480021016000F02D
:1041200019FB6C46CDE9000120460221FFF724FE71
:1041300003492046FFF73AFEDCBD00BF047502408C
:104140003F000000E0B502AF00F004FB6C46CDE993
:10415000000120460021FFF70FFE03492046FFF72C
:1041600025FE00F07FFBFEDE44000000DCB504AF5E
:1041700000F0F0FA6C46CDE9000120460421FFF77B
:10418000FBFD0D492046FFF711FE0C4801680906AA
:1041900011D00021016000F0DDFA6C46CDE900018C
:1041A00020460221FFF7E8FD05492046FFF7FEFD06
:1041B000044801210170DCBD5300000000010040F3
:1041C0005400000094F10320F0B503AF2DE9C00BBB
:1041D00000F0C0FA6C46CDE9000120460421FFF74B
:1041E000CBFD5D492046FFF7E1FD5C484FF000083C
:1041F0000168090602D04FF000090FE0014651F8AE
:10420000042F120603D04FF00109084606E050F8CB
:10421000081F090600F095804FF00209C0F80080E1
:1042200000F098FA6E460446CDE900010D4630468E
:104230000321FFF7A1FD4A493046FFF7B7FD288863
:104240000C22411C6FF31F3022543046298045490F
:10425000FFF7ACFDDDE900010A88531C6FF31F3244
:1042600000F802900B80404DA878811ECAB2032A44
:1042700028BF0121C9B271B1012967D12A78002A6A
:10428000114618BF01217ABB98F001022CD10121FF
:104290002970002144E0B8F1000F4FD1B9F1000FAF
:1042A00057D1334849F2753103220160C0F8142117
:1042B000016001212F48016000F04CFA6C46CDE905
:1042C000000120460221FFF757FD2B492046FFF74A
:1042D0006DFD2A4800210078A5F80110C0B2002821
:1042E00018BF0120287029E0687890BB18EA010007
:1042F00024D1B9F1020F2CD10120687000F02AFA04
:104300006C46CDE9000120460221FFF735FD174933
:104310002046FFF74BFD2978A878B1FA81F14909C9
:1043200060B159B9687848B10420A870002028808D
:10433000BDE80C0BBDE8F040FFF7BCBDBDE80C0BC1
:10434000F0BD4FF003094FF001088CE7FFF72EFE98
:10435000FEDEFFF749FDFEDE4F0000001C010040BD
:10436000020000005200000022F203205100000071
:1043700000EC0640007502405000000094F103205C
:1043800007484FF4803101604FF48051C0F83C126F
:104390004FF4807103480160034800F007B800BF84
:1043A00004B300400C0500503A140000D0B502AF31
:1043B000002201230021012A05D0845C013203FA86
:1043C00004F42143F7E709B101480160D0BD00BF03
:1043D00000E100E0B0B502AF154D0024B4F5C67F92
:1043E00004D0281900F036F88434F7E711480F217B
:1043F00001234160082101600F4981608121C16072
:104400000E490A6863F302020A6040F202214FF487
:10441000822281620A49C162002101630949425036
:1044200009490A4A42500A48BDE8B040FFF7BEBFFA
:1044300040C103200C150040080000066C16004027
:1044400021100100F4FCFFFFF8FDFFFF0940040804
:104450003B14000009490A69026051E8043F934295
:1044600007D141E80402002A1A4608BF00F0FFB94C
:10447000F2E7BFF32F8F1A46EEE700BF98F1032053
:10448000BCB504AF4FF080400125056000F062F933
:104490006C46CDE9000120460221FFF76DFC05497D
:1044A0002046FFF783FC044805600448BDE8BC4093
:1044B000FFF77CBF55000000040300403C140000DF
:1044C000B0B502AF0C4D0024B4F5C67F04D0281956
:1044D000FFF7C0FF8434F7E70848012101604FF47B
:1044E000607101600648074901600748FFF75EFFF9
:1044F000064880210160B0BD04F0032004030040A1
:10450000047302402194C0013C14000004E100E067
:10451000007800F07F02052A1ED00A281ED00F283E
:104520001ED014281ED019281ED01E281ED02328C5
:104530001ED028281ED02D281ED032281ED0372865
:104540001ED03C281ED041281ED046281ED04B2805
:104550000CBF134A114A1AE01F4A18E01D4A16E020
:104560001B4A14E0194A12E0174A10E0154A0EE0FF
:10457000134A0CE0114A0AE00F4A08E00D4A06E02F
:104580000B4A04E0094A02E0074A00E0054AD1E983
:104590000601CB6811460222184700BF5B140000D9
:1045A0003D1400003F1400004114000043140000BB
:1045B0004514000047140000491400004B1400008B
:1045C0004D1400004F14000051140000531400005B
:1045D000551400005714000059140000014801212F
:1045E0000160704704100040BCB504AF0A4804687D
:1045F00000F0B0F86D46CDE9000128460321FFF731
:10460000BBFB06492846FFF7D1FB2046294600F0B0
:1046100007F8204602B0B0BD501500406000000011
:10462000F0B503AF4DF804BD0C460546D1E90001D5
:104630000C260A88531C6FF31F32865420460B80C9
:104640001449FFF7B3FB05F00F010820DFE801F084
:10465000070D0F091521212121110B131600002030
:104660000CE003200AE0062008E0012006E002201A
:1046700004E0052002E0072000E00420D4E9001255
:1046800013885C1C6FF31F33C85414805DF804BB9F
:10469000F0BDFEDE5F000000E0B502AF00F05AF8AA
:1046A0006C46CDE9000120460021FFF765FB034978
:1046B0002046FFF77BFB00F0D5F8FEDE3E00000051
:1046C000E1B3F0B503AF2DE90007DFF8749082463F
:1046D0000C46B9F80650B9F80400401B00F580708C
:1046E000010424D080B2A04238BF044654FA85F0B9
:1046F000E9B280B2B0F5807F0FD9D9F80080C1F55A
:10470000807608EB01005146324600F051F9A01BBB
:104710000AEB060182B2404604E0D9F800002246C6
:104720000844514600F044F92819A9F80600054844
:1047300080210160BDE80007BDE8F040704700BF80
:10474000ACF1032004E200E080B56F4600F08AF887
:10475000FEDED4D4064905480968C9B200290549D6
:1047600018BF00F5805018BF0231704700D00320F9
:1047700004ED00E090F103202AB110F8013B013A6A
:1047800001F8013BF8E77047F0B503AF4DF804BD01
:10479000D6B201F00104C1F30745D7E90212062E93
:1047A00011D00A2E20D1012D08BF002C1CD11204DB
:1047B0001AD18AB2FF2A17D80171002183700170C3
:1047C000190A417014E0012D0ED16CB18CB2FF2C8E
:1047D0000AD803F47F44B4F5085F05D101710121C3
:1047E00042804370017003E000218180022101605A
:1047F0005DF804BBF0BD024680B2FF2801D900215C
:1048000007E0C2F30310002128B1082801D10120DC
:1048100002E002207047002002F00F017047D4D45C
:104820004FF0FF3151FA80F10C200A2918D8DFE847
:1048300001F006080A0C0E101214171716000120BA
:1048400070470220704703207047042070470520FE
:1048500070470620704707207047082070470B20DC
:104860007047FFBEAABE62B6704772B6704740BFBF
:10487000704720BF7047F0B503AF4DF8048DA2B369
:10488000531E02F0030C032B14D20022BCF1000FC4
:104890002BD08B5CBCF1010F835426D0531CBCF190
:1048A000020FCE5CC65420D00232895C81545DF880
:1048B000048BF0BDACEB020E01F10108441C6FF05B
:1048C000030208EB0206A5180432F378EB70337983
:1048D0002B7173796B71B379AB710EEB02030433F7
:1048E000EFD10432BCF1000FD3D15DF8048BF0BDE1
:1048F000D0B502AF12B3531E02F0030C032B01D24A
:1049000000220FE0ACEB020E421C6FF00303D41840
:104910000433A17161712171E1700EEB0304043461
:10492000F5D11A1DBCF1000F1ABF8154BCF1010F63
:10493000D0BD0244BCF1020F517000D1D0BD9170C6
:10494000D0BDF0B503AF2DE9000B4AB3A2F1010EC3
:10495000C2F1000C0023CC5CC55CA54224D19E456D
:104960001ED001EB030800EB030998F8014099F809
:104970000150A54218D10CEB0306B41C10D098F8D6
:10498000024099F80250A5420ED1F41C08D098F8C4
:10499000034099F80350A54206D104339A42DAD174
:1049A0000020BDE8000BF0BD281BBDE8000BF0BDEA
:1049B000FFF761BF042A38BFFFF7FABFB0B502AFF7
:1049C000A2F1040C012303EB9C0313F003030ED0AC
:1049D0008E4604465EF8045B012B44F8045B1FD14D
:1049E000634620467146BCF10C0F04D212E0134618
:1049F000BCF10C0F0ED30D68103B0560032B4D6806
:104A000045608D688560CD6801F11001C56000F1D9
:104A10001000F0D802F00302BDE8B040FFF7C8BFB5
:104A20004D68022B456007D1A2F108030831083018
:104A3000BCF10C0FDFD2EDE78B680C318360A2F183
:104A40000C030C30BCF10C0FD5D2E3E70B4611463A
:104A50001A46FFF74DBF1346D2B2042938BFFFF7FD
:104A6000F5BFD0B502AFA1F1040E42EA0363012401
:104A700043EA024304EB9E0443EA022314F00304D6
:104A800010D08446012C4CF8043B10D1744660468B
:104A9000BEF10C0F1ED201F00301BDE8D04060460C
:104AA000FFF7D4BF0C46BEF10C0F13D2F3E7022C74
:104AB000436007D10830A1F108048446BEF10C0F11
:104AC00008D2E8E783600C30A1F10C048446BEF103
:104AD0000C0FE0D3C0E90033103CC0E902331030C2
:104AE000032CF7D8844601F00301BDE8D0406046AE
:0A4AF000FFF7ACBF0022FFF7AEBFD6
:104AFC00C144000081440000D54300008143000004
:104B0C0040C003200000000012010002EF0201402F
:104B1C002020100300010000000109024B000201DB
:104B2C000080FA080B0002020201000904000001D7
:104B3C0002020100052400100105240103010424D4
:104B4C000202052406000107058103400020090428
:104B5C000100020A000000070502024000000705E0
:104B6C008202400000000000A120000000000200B2
:104B7C000300000001000000028025000000000876
:040000030000277D55
:00000001FF
